:1000000012C02CC02BC02AC029C028C027C026C0BF
:1000100025C025C023C022C021C020C01FC01EC0D3
:100020001DC01CC01BC011241FBECFE5D4E0DEBF25
:10003000CDBF11E0A0E6B0E0ECECF6E102C0059027
:100040000D92A037B107D9F711E0A0E7B1E001C0E8
:100050001D92A73AB107E1F744D336CBD1CF1F9217
:100060000F920FB60F9211242F933F934F935F93EC
:100070006F937F938F939F93AF93BF93EF93FF9370
:10008000C4DAFF91EF91BF91AF919F918F917F91D2
:100090006F915F914F913F912F910F900FBE0F90F5
:1000A0001F90189581E06FE0AAD90895880F8E7788
:1000B000A6D90895880F8E778068CDD9089587E3F3
:1000C000F9DF80937B0108950F931F93082F162F5C
:1000D000F1DF000F10951823802F8E77612F8FD9B5
:1000E0001F910F91089584E163E0EEDF08950F936F
:1000F0001F93182F062FDEDF110F082B812F8E770D
:10010000602F7DD91F910F910895DF92EF92FF929A
:100110000F931F93CF93DF93182F092FD62E7A01B9
:1001200085E064E0D1DF8AE060E8E1DF212F302F55
:10013000C901EC0110E004C082E1699160D91F5F40
:100140001D15D0F382E063E05AD91FEF85E0B2DFDE
:10015000115011F082FFFACF82E2ACDFF701808309
:1001600081E2A8DFF7018183DF91CF911F910F9189
:10017000FF90EF90DF9008954F925F926F927F9281
:100180008F929F92AF92BF92CF92DF92EF92FF92A7
:100190000F931F93DF93CF930F92CDB7DEB7D82E77
:1001A0005B01F42E390148018CE0D81659F0EEE0DD
:1001B000DE1619F0CC24EE2409C0F2E1CF2EE0E1E6
:1001C000EE2E04C077E7C72E60E3E62E6C2D606844
:1001D00084E015D984E060E877DF8AE060E887DFB3
:1001E00082E060E00CD900E010E04F2C552408C0FC
:1001F000F501E00FF11F82E1608101D90F5F1F4F10
:1002000004151505A8F382E06D2DF9D8FCE0DF1682
:1002100019F48DE060E86BDF00ED17E084E04ADF61
:10022000F82E0150104021F080FD02C08E21B1F364
:100230008DE060E849DF012B09F445C086E03ADF34
:100240008B7109F040C0FC2081E0F822ECE0DE1662
:10025000E1F58AE02FDF982F8CE099832BDF877000
:100260009981292F30E0882351F02150304053E00C
:10027000220F331F5A95E1F7280F311D05C043E0C7
:10028000220F331F4A95E1F7F4013183208399232C
:1002900011F491E003C0913108F090E100E010E02A
:1002A000C92EDD240CC089E005DFF301E00FF11F4A
:1002B0008083F801E557FE4F80830F5F1F4F0C15B9
:1002C0001D0588F302C082E0F82E8F2D0F90CF918C
:1002D000DF911F910F91FF90EF90DF90CF90BF9033
:1002E000AF909F908F907F906F905F904F90089508
:1002F0000F931F93DF93CF93CDB7DEB72B970FB636
:10030000F894DEBF0FBECDBF23E92B8320E72C83FB
:10031000DC01FE0135968E010D5F1F4F9E01265FA9
:100320003F4F8D918193E217F307D9F7C80167E03A
:10033000AF01EBDE8CE0B80149E098018E010F5F60
:100340001F4F1ADF882331F489819A81489711F46D
:100350008B8101C080E02B960FB6F894DEBF0FBEF4
:10036000CDBFCF91DF911F910F910895CF92DF9272
:10037000EF92FF920F931F93DF93CF93CDB7DEB72A
:1003800064970FB6F894DEBF0FBECDBF6B0190EA45
:100390009B838C83A3E0EA2EF12CEC0EFD1EC7019B
:1003A00062E0AE014B5F5F4FB0DE8CE0B70144E02E
:1003B00097018E010F5F1F4FDFDE882389F589814A
:1003C0009A81049769F58B818F708A3049F520E016
:1003D00030E08701F801E20FF31FD601A20FB31F2F
:1003E0008C9180832F5F3F4F2031310599F7C801F1
:1003F00060E1AE014D5E5F4F88DE8CE0B80142E106
:1004000098018E010F5F1F4FB7DE282F882341F41C
:1004100089819A81049721F48B818F708A3009F049
:1004200022E0822F64960FB6F894DEBF0FBECDBFD8
:10043000CF91DF911F910F91FF90EF90DF90CF90C0
:1004400008950F931F93DF93CF9300D0CDB7DEB7FE
:100450008B0190E3FB0190838183AB014E5F5F4F83
:10046000CB0162E052DE8CE0B80144E098018E01DD
:100470000F5F1F4F81DE282F882329F489819A81FD
:100480008039910509F022E0822F0F900F90CF91D3
:10049000DF911F910F9108950F931F93DF93CF93D7
:1004A0000F92CDB7DEB78C01198280EEF801808300
:1004B00080E58183A8014E5F5F4FC80162E070E074
:1004C00024DE8CE0B80144E098018E010F5F1F4FDD
:1004D00053DE0F90CF91DF911F910F910895EF920E
:1004E000FF920F931F93DF93CF9300D0CDB7DEB76A
:1004F0007C018AE160E083D785E9F701808380E2AF
:1005000081838CE0B70142E097018E010F5F1F4F9E
:1005100033DE482F882389F490E020E030E0F701B3
:10052000E20FF31F808198272F5F3F4F2430310562
:10053000B1F7F7018481981342E0842F0F900F9058
:10054000CF91DF911F910F91FF90EF900895EF925F
:10055000FF920F931F93DF93CF9300D0CDB7DEB7F9
:100560007C018AE160E04BD783E9F701808380E278
:1005700081838CE0B70142E097018E010F5F1F4F2E
:10058000FBDD482F882389F490E020E030E0F7017C
:10059000E20FF31F808198272F5F3F4F24303105F2
:1005A000B1F7F7018481981342E0842F0F900F90E8
:1005B000CF91DF911F910F91FF90EF900895FF92DF
:1005C0000F931F93DF93CF9300D0CDB7DEB7F82EF4
:1005D0008B018AE167E013D7F801F0828CE0B80163
:1005E00041E098018E010F5F1F4FC6DD282F882341
:1005F00021F489819A81409709F022E0822F0F909F
:100600000F90CF91DF911F910F91FF9008950F935D
:100610001F93DF93CF93CDB7DEB72E970FB6F89425
:10062000DEBF0FBECDBFD9018B836C838E010B5F04
:100630001F4F9E012D5F3F4FBE01655F7F4FFA0147
:100640008191AF01F80181938F01E617F707B9F7A0
:100650008C918B8711968C9111978C8712968C9127
:1006600012978D8713968C918E878EE0B9014CE09E
:100670008E010F5F1F4F80DD182F882319F488E04B
:1006800019DD83FF12E0812F2E960FB6F894DEBF9E
:100690000FBECDBFCF91DF911F910F91089584E1DF
:1006A00009DD90E083709070892B19F484E163E098
:1006B0001EDD089581E06FE0A2D684E56DE89FD647
:1006C00086E56EE39CD688E56EE199D68AE560E022
:1006D00096D68AE260E493D682E26DE390D6DFDFBD
:1006E0000895EF92FF920F931F93DF93CF93CDB7AF
:1006F000DEB760970FB6F894DEBF0FBECDBF0FD642
:1007000079D67CD7D7DFB89AC09883B7856083BF86
:1007100089B7816089BF12BE80E090E0C0D7809326
:100720009D0181E090E0BBD780939E0182E090E044
:10073000B6D780939F0183E090E0B1D78093A0016A
:1007400084E090E0ACD78093A10185E090E0A7D74A
:100750008093810186E090E0A2D78093820187E0B8
:1007600090E09DD78093830188E090E098D78093B4
:10077000840189E090E093D7809385018AE090E03E
:100780008ED7809386018BE090E089D78093870194
:100790008CE090E084D7809388018DE090E07FD753
:1007A000809389018EE090E07AD780938A018FE070
:1007B00090E075D78093A20180E190E070D780939C
:1007C000A30181E190E06BD78093A40182E190E0E6
:1007D00066D78093A50183E190E061D78093A6015D
:1007E00084E190E05CD78093760185E190E057D773
:1007F0008093770186E190E052D78093780187E17A
:1008000090E04DD78093790188E190E048D78093BC
:100810007A0181E078D580EA9FE00197F1F778943A
:1008200016D780937001843009F0FDC381E06BD549
:1008300080EA9FE00197F1F70AD780937001843036
:1008400061F481E060D580EA9FE00197F1F77E01D5
:100850000894E11CF11C01E0A3C0813009F44DC3F0
:10086000823009F07EC081E04ED580EA9FE001979A
:10087000F1F780E090E060E01AD781E090E060E07E
:1008800016D782E090E060E012D783E090E060E06D
:100890000ED784E090E060E00AD785E090E060E069
:1008A00006D786E090E060E002D787E090E060E065
:1008B000FED688E090E060E0FAD689E090E060E063
:1008C000F6D68AE090E060E0F2D68BE090E060E05F
:1008D000EED68CE090E060E0EAD68DE090E060E05B
:1008E000E6D68EE090E060E0E2D68FE090E060E057
:1008F000DED680E190E060E0DAD681E190E060E071
:10090000D6D682E190E060E0D2D683E190E060E06C
:10091000CED684E190E060E0CAD685E190E060E068
:10092000C6D686E190E060E0C2D687E190E060E064
:10093000BED688E190E060E0BAD681ECE4D480E6EF
:1009400090E01DD588E293E228EC30E0F901319780
:10095000F1F70197D9F781E0D6D480EA9FE00197BB
:10096000F1F7ADDB81E8CFD483E790E008D581ECE7
:10097000CAD485E890E003D580917B01813919F4D0
:100980008FE890E0FCD480917B01823919F483E9EF
:1009900090E0F5D485EDB7D487E990E0F0D44CCF62
:1009A00056D680937001843061F481E0ACD480EA43
:1009B0009FE00197F1F77E010894E11CF11C01E032
:1009C00093C0813009F499C280E89DD489EA90E00F
:1009D000D6D486E2B701F3DD882361F580EC93D4A9
:1009E00081EB90E0CCD480918B01843049F48091EC
:1009F0008C01882329F487EB90E0C1D41092730115
:100A000080918B01823049F480918C01882329F4F4
:100A10008CEB90E0B4D41092730180918B018434FC
:100A200049F480918C01882329F481EC90E0A7D4CB
:100A300000937301C7018BDDACE7B1E0F70195E0EE
:100A400001900D929150E1F78823B9F584E95BD4C8
:100A50008DEC90E094D480917C0190E06CD58091F5
:100A60007D0190E068D580917E0190E064D5809111
:100A70007F0190E060D58091800190E05CD580E0BE
:100A800090E060917C0113D681E090E060917D015F
:100A90000ED682E090E060917E0109D683E090E07E
:100AA00060917F0104D684E090E060918001FFD5E1
:100AB0008AED29D482ED90E062D48CE791E018DCD5
:100AC000182F882309F46CCF80917301813009F4C9
:100AD00067CF8AEC18D4812F8695869586958BD51D
:100AE00089ED90E04CD45CCFB2D580937001843016
:100AF00061F481E008D480EA9FE00197F1F77E017C
:100B00000894E11CF11C01E093C0813009F4F5C1A7
:100B100080E8F9D38DED90E032D486E2B7014FDD65
:100B2000882361F580ECEFD381EB90E028D48091AD
:100B30008B01843049F480918C01882329F487EB60
:100B400090E01DD41092730180918B01823049F4A2
:100B500080918C01882329F48CEB90E010D41092C2
:100B6000730180918B01843449F480918C01882336
:100B700029F481EC90E003D400937301C701E7DC12
:100B8000ACE7B1E0F70195E001900D929150E1F7EB
:100B90008823B9F584E9B7D38DEC90E0F0D3809148
:100BA0007C0190E0C8D480917D0190E0C4D4809114
:100BB0007E0190E0C0D480917F0190E0BCD4809110
:100BC000800190E0B8D485E090E060917C016FD521
:100BD00086E090E060917D016AD587E090E06091C9
:100BE0007E0165D588E090E060917F0160D589E065
:100BF00090E0609180015BD58AED85D382ED90E035
:100C0000BED38CE791E074DB182F882309F46CCFF6
:100C100080917301813009F467CF8AEC74D3812FFE
:100C2000869586958695E7D485EE90E0A8D35CCF2F
:100C30000ED580937001843061F481E064D380EA42
:100C40009FE00197F1F77E010894E11CF11C01E09F
:100C500093C0813009F451C180E855D38CEE90E007
:100C60008ED386E2B701ABDC882361F580EC4BD3F1
:100C700081EB90E084D380918B01843049F48091A2
:100C80008C01882329F487EB90E079D310927301CB
:100C900080918B01823049F480918C01882329F462
:100CA0008CEB90E06CD31092730180918B018434B3
:100CB00049F480918C01882329F481EC90E05FD382
:100CC00000937301C70143DCACE7B1E0F70195E0A5
:100CD00001900D929150E1F78823B9F584E913D37F
:100CE0008DEC90E04CD380917C0190E024D48091F5
:100CF0007D0190E020D480917E0190E01CD4809111
:100D00007F0190E018D48091800190E014D48AE0B3
:100D100090E060917C01CBD48BE090E060917D010C
:100D2000C6D48CE090E060917E01C1D48DE090E06B
:100D300060917F01BCD48EE090E060918001B7D4D7
:100D40008AEDE1D282ED90E01AD38CE791E0D0DA1F
:100D5000182F882309F46CCF80917301813009F436
:100D600067CF8AECD0D2812F86958695869543D41D
:100D700085EE90E004D35CCF6AD480937001843018
:100D800061F481E0C0D280EA9FE00197F1F77E0133
:100D90000894E11CF11C01E093C0813009F4ADC05E
:100DA00080E8B1D284EF90E0EAD286E2B70107DCB6
:100DB000882361F580ECA7D281EB90E0E0D28091AE
:100DC0008B01843049F480918C01882329F487EBCE
:100DD00090E0D5D21092730180918B01823049F45A
:100DE00080918C01882329F48CEB90E0C8D210927A
:100DF000730180918B01843449F480918C018823A4
:100E000029F481EC90E0BBD200937301C7019FDB12
:100E1000ACE7B1E0F70195E001900D929150E1F758
:100E20008823B9F584E96FD28DEC90E0A8D2809147
:100E30007C0190E080D380917D0190E07CD3809113
:100E40007E0190E078D380917F0190E074D380910F
:100E5000800190E070D38FE090E060917C0127D416
:100E600080E190E060917D0122D481E190E0609189
:100E70007E011DD482E190E060917F0118D483E16E
:100E800090E06091800113D48AED3DD282ED90E034
:100E900076D28CE791E02CDA182F882309F46CCFF6
:100EA00080917301813009F467CF8AEC2CD2812FB5
:100EB0008695869586959FD385EE90E060D25CCF2F
:100EC000C6D3809370018430B1F481E01CD280EAF3
:100ED0009FE00197F1F784EC16D28CEF90E04FD2AF
:100EE00088E293E228EC30E0F9013197F1F70197BD
:100EF000D9F781E002C0813031F405D280EA9FE069
:100F00000197F1F790C080E8FED186E091E037D2FA
:100F100086E2B70154DB882361F580ECF4D181EBE4
:100F200090E02DD280918B01843049F480918C0126
:100F3000882329F487EB90E022D2109273018091EC
:100F40008B01823049F480918C01882329F48CEB49
:100F500090E015D21092730180918B01843449F492
:100F600080918C01882329F481EC90E008D20093D1
:100F70007301C701ECDAACE7B1E0F70195E001904D
:100F80000D929150E1F78823B9F584E9BCD18DEC3D
:100F900090E0F5D180917C0190E0CDD280917D01EF
:100FA00090E0C9D280917E0190E0C5D280917F010E
:100FB00090E0C1D28091800190E0BDD284E190E0C8
:100FC00060917C0174D385E190E060917D016FD3E5
:100FD00086E190E060917E016AD387E190E06091C4
:100FE0007F0165D388E190E06091800160D38AED54
:100FF0008AD182ED90E0C3D18CE791E079D9182FA6
:10100000882309F45DCF80917301813009F458CFB2
:101010008AEC79D1812F869586958695ECD285EEDE
:1010200090E0ADD14DCF80EC6ED18EE091E0A7D1B4
:1010300086E28E010F5F1F4FB801C1DA882309F0E5
:10104000EFCB81E060D180EA9FE00197F1F7C80122
:101050007EDAACE7B1E0F80195E001900D92915095
:10106000E1F7882309F0DCCB90917C0180919D0110
:10107000981781F590917D0180919E01981751F507
:1010800090917E0180919F01981721F590917F01A9
:101090008091A0019817F1F4909180018091A101B5
:1010A0009817C1F482E82FD182E291E068D182ECF6
:1010B0002AD189EA90E063D181E080937201C09ADD
:1010C00080E593EC28EC30E0F9013197F1F70197D6
:1010D000D9F7C09890917C0180918101981781F592
:1010E00090917D0180918201981751F590917E0138
:1010F00080918301981721F590917F01809184015F
:101100009817F1F490918001809185019817C1F4AE
:1011100082E8F9D082E291E032D182ECF4D08DED18
:1011200090E02DD181E080937201C09A80E593EC2C
:1011300028EC30E0F9013197F1F70197D9F7C09821
:1011400090917C0180918601981781F590917D01A5
:1011500080918701981751F590917E0180918801C7
:10116000981721F590917F01809189019817F1F4EA
:101170009091800180918A019817C1F482E8C3D0D0
:1011800082E291E0FCD082ECBED08CEE90E0F7D011
:1011900081E080937201C09A80E593EC28EC30E006
:1011A000F9013197F1F70197D9F7C09890917C0137
:1011B0008091A201981781F590917D018091A30102
:1011C000981751F590917E018091A401981721F50F
:1011D00090917F018091A5019817F1F49091800181
:1011E0008091A6019817C1F482E88DD082E291E047
:1011F000C6D082EC88D084EF90E0C1D081E08093AB
:101200007201C09A80E593EC28EC30E0F901319747
:10121000F1F70197D9F7C09890917C018091760100
:10122000981781F590917D0180917701981751F57C
:1012300090917E0180917801981721F590917F011E
:10124000809179019817F1F49091800180917A0151
:101250009817C1F482E857D082E291E090D082ECF6
:1012600052D086E091E08BD081E080937201C09AE9
:1012700080E593EC28EC30E0F9013197F1F7019724
:10128000D9F7C09880917201882371F482EC3BD029
:1012900081E391E074D088E39AE428EC30E0F9012E
:1012A0003197F1F70197D9F781E02DD080EA9FE0DF
:1012B0000197F1F710927201B3CA9AE69A95F1F785
:1012C000909892B3807F9F70982B92BB929A85E002
:1012D0008A95F1F79298089592B3282F207F9F70F6
:1012E000292B22BB929A25E0922F9A95F1F792989A
:1012F00092B38295807F9F70982B92BB929A2A9589
:10130000F1F7929808959AE69A95F1F79098E4DFAC
:1013100008959AE69A95F1F7909ADEDF08950F9373
:101320001F9381B3806F81BB889A899A8A9A80E9DA
:1013300091E028EC30E0F9013197F1F70197D9F706
:1013400080E3BBDF80E29EE40197F1F780E3B5DF45
:1013500000EA1FE0C8010197F1F780E3AEDF88E201
:10136000ACDF88E2D0DF8CE0CEDF81E0CCDFC801EB
:101370000197F1F786E0C7DF1F910F910895CF9392
:10138000DF93EC0102C02196C4DF88818823D9F75E
:10139000DF91CF910895CF93DF93EC0104C0FE015C
:1013A00084912196B6DF88818823C9F7DF91CF9198
:1013B00008950F931F93CF93DF938C01862F90E0B6
:1013C0008770907023E0880F991F2A95E1F7806459
:1013D0009ADFC0E0D0E0F801EC0FFD1FE4918E2F02
:1013E00098DF2196C830D105B1F7DF91CF911F91D9
:1013F0000F91089584E387BB8CE388BB0895C5985B
:10140000C29820E031E087FF02C0C49A01C0C498AE
:10141000C59A932F9A95F1F7C598932F9A95F1F75E
:101420002F5F283011F0880FEECF90E021E067FFAA
:1014300002C0C49A01C0C498C59A822F8A95F1F758
:10144000C598822F8A95F1F79F5F983011F0660F4B
:10145000EECFC29A0895382FC598C29880E020E058
:1014600041E037FF02C0C49A01C0C498C59A942FC6
:101470009A95F1F7880FB3998160C598942F9A9542
:10148000F1F72F5F283011F0330FEBCF20E031E080
:10149000880FB3998160C59A932F9A95F1F7C598F3
:1014A000932F9A95F1F72F5F283091F7C29A0895FC
:1014B000EF92FF920F931F939C0168EE73E0DBD0D5
:1014C000182F092FC90168EE73E0D5D0662311F4F7
:1014D00080E302C0862F805D1CDF812F902F64E6A1
:1014E00070E0C9D0F82EE92E812F902F64E670E0CD
:1014F000C2D0662311F480E302C0862F805D09DF2D
:101500008F2D9E2D6AE070E0B6D0362F8F2D9E2D48
:101510006AE070E0B0D0182F332311F480E302C0EA
:10152000832F805DF6DE812F805DF3DE1F910F91AA
:10153000FF90EF9008950F931F939C0164E670E075
:101540009AD0182F092FC90164E670E094D0662361
:1015500011F480E302C0862F805DDBDE812F902FA7
:101560006AE070E088D0362F812F902F6AE070E01B
:1015700082D0182F332311F480E302C0832F805DC3
:10158000C8DE812F805DC5DE1F910F9108951F93E6
:10159000282F64E664D0192F822F61D0882311F49C
:1015A00080E301C0805DB5DE812F6AE058D0282F2E
:1015B000812F55D0192F222311F480E302C0822FEE
:1015C000805DA7DE812F805DA4DE1F9108951F93AB
:1015D000282F6AE044D0382F822F41D0192F33238F
:1015E00011F480E302C0832F805D93DE812F805D44
:1015F00090DE1F910895805D8CDE089584B3807F16
:1016000084BB85B38F6085BB0895989902C091E033
:101610000BC09A9902C093E007C0999902C092E06A
:1016200003C09B9911C094E080917501873420F02C
:101630008EE38093750105C08F5F809375018430C0
:1016400029F4909374010895109275010895809182
:101650007401109274010895809374010895991B88
:1016600079E004C0991F961708F0961B881F7A9599
:10167000C9F780950895AA1BBB1B51E107C0AA1F9B
:10168000BB1FA617B70710F0A61BB70B881F991F23
:101690005A95A9F780959095BC01CD010895E199DF
:1016A000FECF9FBB8EBBE09A99278DB30895262F5E
:1016B000E199FECF9FBB8EBB2DBB0FB6F894E29A8B
:0C16C000E19A0FBE01960895F894FFCF48
:1016CC004D656D6F727920697320636C656172650D
:1016DC00642100524649442D5243353232206D6FFD
:1016EC0064756C6500536F66747761726520005683
:1016FC002E3100562E32004361726473206C65618A
:10170C00726E696E67203E3E004361726420233125
:10171C0000436172643A0020533530002053373057
:10172C000020556C7472614C696768740049443AC6
:10173C00200053617665642100204B620043617286
:10174C006420233200204B6279746500436172641B
:10175C00202333004361726420233400436F6D7087
:10176C006C657465640043617264202335003C3CF5
:10177C002061747461636820612063617264203E2F
:10178C003E00416C6C6F77656420616363657373B5
:10179C00004163636573732044656E696564210061
:1017AC00FFFFFFFFFFFF0000000000000000000033
:1017BC00A0A1A2A3A4A5000000000000000000004E
:1017CC00D3F7D3F7D3F700000000000000000000AF
:00000001FF
